:020000020000FC
:100000000C944F000C9400000C944B010C940000D5
:100010000C9400000C9400000C9400000C94000060
:100020000C9400000C94C8000C9400000C94000088
:100030000C9400000C947D000C94B8000C9400000B
:100040000C9400000C9400000600020001008701DF
:100050000200900125642044656720460025642045
:1000600044656720430025642044656720460A00F4
:1000700043757272656E742054656D703A00102776
:10008000E80364000A0001000010000110000100F4
:100090008B01020080C048004E0090000000F894E0
:1000A000EE27ECBBE5BFF8E1F1BDF0E1F1BD8DE07D
:1000B000A2E0BB27ED938A95E9F780E094E0A0E603
:1000C000ED930197E9F7E6E9F0E005901590BF019F
:1000D000F001309751F0A591B591859195910590DA
:1000E0000D920197E1F7FB01F0CFEFE5EDBFE4E002
:1000F000EEBFCFE5D1E00C945C010E947D03CA14F1
:10010000DB0451F0EC2DFD2D3196CE2EDF2E3197F4
:10011000E159FE4FE081ECB90E948B031895AA24A7
:10012000BB24E1E0F0E0CE2EDF2E0E944903EDE09B
:10013000EC930E944903EAE0EC93A881B981EC9129
:10014000E03089F0EA2DFB2D3196AE2EBF2E31978F
:10015000E159FE4FFF93EF93ED91A883B983AF91DF
:10016000BF91EC93EACFE0916F01ECB9229608952C
:100170000E947D0344B055B0A42DB52DE0E4F0E01D
:100180000E94B8034E2E5F2E369A0E948B0318955C
:100190000E947D03EE27E2BFE82DF92D31968E2EC9
:1001A0009F2EA0918701B0918801EA17FB0711F0FB
:1001B0000C944801E1E0F0E0E615F70529F5E42D9F
:1001C000F52D662777270E943904DF01CB01EAEA83
:1001D000F1EF62E070E40E94F204E0938301F09397
:1001E000840160938501709386010E9413044E2E52
:1001F0005F2EE0E6F1E0FA93EA93E4E5F0E00E9496
:10020000530384E00E945C03062C072869F5E0E6AE
:10021000F1E0FA93EA93EDE5F0E0FA93EA93E42D46
:10022000F52DDF01CB01882799270E94E003E8E440
:10023000F1EE6AEF7FE30E94C004DF01CB01E0E052
:10024000F0E060E072E40E94E3030E947004DF01CA
:10025000CB01E6E6F6E666EE7FE30E94F2040E943A
:10026000D90384E00E945C03E0E6F1E0FA93EA93AC
:10027000E6E6F0E00E94530384E00E9481022896A3
:10028000E0E6F1E0FA93EA930E948F008824992433
:100290000E948B0318950E947D03E62DF72D319661
:1002A0006E2E7F2EE2E0F0E0E615F70511F46624ED
:1002B00077240E948B031895EFEFE7BBE0EAE1BBE0
:1002C000E8E5EAB9E7E1E9B9E0E1EA930E942C0345
:1002D000EE27EA93EA930E94D002E0E7F0E0FA9377
:1002E000EA930E941C03E0E2E7B9EEECE6B9E3E032
:1002F000E3BFEE27E2BFE1E0E9BFE0ECEBBFEAE0FD
:10030000E5BF7894FFCFFFCF5F9BFECFECB10895A0
:100310005D9BFECFE881ECB921960895E0918901BB
:10032000F0918A01309769F0A0918901B0918A011A
:100330001196A0938901B0938A011197E881EC93FB
:1003400004C0E881EA930E948801219608952697C7
:100350000E94330500E0EE85FF853196EE87FF872A
:100360003197E4912E2FE03011F40C947D02E02FB0
:10037000E03041F4253211F401E003C02A930E94D9
:100380008E01BAC0E13099F4253229F42A930E94F3
:100390008E0100E0B1C002E030E010E02B3211F439
:1003A0003BE2AAC0203211F430E2A6C002C0E23023
:1003B00031F4203319F4106105E09EC004C0E5302B
:1003C00011F00C947C02E22FE33639F40E946B03A7
:1003D000EC91EA930E948E018EC0E33799F40E945B
:1003E0006B030E94CF03EE83FF83AE81BF81ED914B
:1003F000AE83BF832E2FE03021F02A930E948E011E
:10040000F4CF79C0E037A9F40E946B030E94CF03B8
:10041000E887F987E885F9853196E887F987319784
:10042000E4912E2FE03021F02A930E948E01F2CF2A
:1004300062C0E43611F0E93611F4116002C0E5370C
:1004400019F4EEE7F0E00AC0E83511F4126004C0D8
:10045000E83711F00C947B02E8E8F0E0E887F987D0
:1004600010FF14C00E946B034D915C9140505040AE
:100470003CF4E42FF52F0E949D034E2F5F2F3DE2A9
:10048000303019F03A930E948E0104C00E946B0331
:100490004D915C9120E3E885F9853296E887F987EC
:1004A00032970E94D503EA87FB874E175F0720F03B
:1004B0002F5F4E1B5F0BC9F714FD09C0E0E3E21785
:1004C00030F0AA85BB85A130E0E0BE0761F4106181
:1004D000E9E3E21728F411FF02C0295F01C0295D9A
:1004E0002A930E948E01AA85BB85E1E0F0E0EA171D
:1004F000FB0708F4CFCF00E02ECF0E943A056096AC
:100500000895F82E2297DE0112970E949903A8837E
:10051000B983DE0114960E9499030E94CB03E093F5
:100520008901F0938A01DE0112960E9499030E94CC
:10053000CB03FA93EA93EA81FB81FA93EA930E9450
:10054000A701A0918901B0918A01EE27EC93229630
:100550000895A4B3AF70A4BBA99AA8980CD0AA9A86
:100560000AD09F99FBCFAA980895A07FAB2BA5BB7B
:10057000AA9A01D0AA980000000000000000000024
:1005800000000895A998A4B3A76FA4BBB5B3BF702A
:10059000A881EBDFA881A295E8DFA99A21960895AA
:1005A0000E94A902E881FF27E557FE4FE081A9815B
:1005B000EA0FEA930E94C202E980E881E0938F018A
:1005C000229608950E94A902ECE00E947203E1E0E5
:1005D000EA930E94C202EE27E0938F01EE2E089567
:1005E000EF93FF93A8816894AA3031F0E894E394E4
:1005F000E0919001EE1568F4E0918F01EF5FE093D8
:100600008F01EE27EA93E0918F01EA930E94D002D6
:100610002EF09FDFA89AA881AA93B4DFFF91EF91F3
:1006200021960895F981E881A191AA2319F0AA934E
:10063000D7DFFACF22960895E881F981C895002086
:1006400021F031960A92CCDFF9CF22960895AA279D
:10065000BB271197F1F70895AA98A898E881E0932D
:100660009001E058E0938D01E881E054E0938E0121
:100670003ED03DD03CD00E942703E0E233D0E8E2F8
:1006800031D0E6E0EA930E94C2020E94E202219683
:100690000895EA2DFB2D3196AE2EBF2E3197E159EC
:1006A000FE4FDF010895FA93EA93E42DF52D6627B6
:1006B00077270E94D90308950E9481022896EE2789
:1006C000EA93E1E0EA930E94D002E0E6F1E0FA93D7
:1006D000EA930C941203AC85BD851497AC87BD8753
:1006E00014960895EA930E94C2020C94A9020E94F3
:1006F0002703E0E3EA930C94C2020A921A92FA9258
:100700006A937A938A939A93AA93BA93EA93FA9301
:100710000FB60A92089509900FBEF991E991B99127
:10072000A9919991899179916991F990199009907C
:1007300008950024AF0DB01D0895E095F095319611
:100740000895E095F09560957095EF5FFF4F6F4FBE
:100750007F4F089566277727F7FF08956FEF7FEFA4
:10076000089588279927B7FF08958FEF9FEF089581
:100770000024112490E1AA0FBB1F001C111C0E1AAB
:100780001F0A18F40E0E1F1E01C0A1609A9599F75A
:10079000FD01D0010895ED91FC9111970895ED911F
:1007A000FD916D917C91139708950590F491E02D42
:1007B00008957A936A93FA93EA930895689401C02E
:1007C000E89401D057D0182E862F612D192E972F1F
:1007D000712D1B2EBF2FF12D1A2EAE2FE12D089556
:1007E00050E8572711F45F93BFC05F3F31F0660FA9
:1007F000000C57956795752F08955F9300200AF0B8
:10080000B9C0ACC050E8192E1522880F991F952742
:10081000550F879550E8072E0522660F771F75271D
:10082000550F679508955F93F5DF703810F07F3F9F
:1008300030F056E1571B0AF49DC0583108F094C0BF
:100840007727583028F0EF2FF62F672F5850F9CF21
:10085000552331F076956795F795E7955A95D1F739
:100860007727002012F435D07FEF5F9108956894C8
:1008700001C0E894309760407040B1F0002426F049
:10088000772312F400945DDF172E7EE1112032F001
:100890007A95EE0FFF1F661F111CF9CFEF2FF62F71
:1008A000612D5F939DDF5F9108955E2FEA2FA52F45
:1008B0005F2FFB2FB52F562F682F852F572F792F9E
:1008C000952F502D012C152E0895EA0FFB1F681F40
:1008D0000895E095F0956095EF5FFF4F6F4F089595
:1008E0005F9390DF903849F150E81526703821F178
:1008F000572F591B13F112F4D8DFFACF583118F0E3
:10090000AA27BB278827583028F0AB2FB82F882775
:100910005850F9CF552329F08695B795A7955A9544
:10092000D9F7502D512562F0D0DF38F46795F7954F
:10093000E795739513F41EC0B8DF52DF5F910895F9
:10094000EA1BFB0B680B81F010F40094C2DF6623F6
:10095000A2F3EE0FFF1F661F7A95CBF7EFEFFFEFC5
:100960006FE77FEF5F910895EE27FF2766277727D0
:100970005F910895EFEFFFEF6FE77FE75F910895D5
:100980005F9340DF703881F3903871F3012408944D
:10099000791F23F44CF300200AF3ECCF3F934F93DD
:1009A000112433274427552798E1330F441F551F3F
:1009B000EE1FFF1F661F30F43A0F4B1F581FE11D3B
:1009C000F11D611D9A9589F74F913F9166232AF099
:1009D000550FEE1FFF1F661F02C07395E3F200DF85
:1009E0005F9108955F930EDF703819F4112012F6AD
:1009F000B5CF903809F4B8CF01240894970B1BF4B5
:100A0000D4F30020F4CF792F6695F795E795869576
:100A1000B795A7954F9311244427552798E1AE1712
:100A2000BF07860728F0AE1BBF0B860B089401C0DA
:100A30008894111C441F551FAA1FBB1F881F9A951D
:100A400071F7E12DF42F652FA695E91FF91F691F96
:100A50004F9166232AF0EE0FFF1F661F7A955BF217
:100A6000BFDE5F9108955A934A933A932A931A935B
:100A70000A9308955D814C813B812A811981088107
:020A80000895D7
:00000001FF
